:1000000001010101010101010101010101010101E0
:1000100001010101010101010101010101010101D0
:1000200001010101010101010101010101010101C0
:1000300001010101010101010101010101000101B1
:1000400001010101010101010101010101010101A0
:100050000101000101010101010001000101010193
:100060000000000000000000000000000000000090
:100070000000000000000000000000000000000080
:100080000000000000000000000000000000000070
:100090000000000000000000000000000000000060
:1000A0000000000000000000000000000000000050
:1000B0000000000000000000000000000000000040
:1000C0000000000000000000000000000000000030
:1000D0000000000000000000000000000000000020
:1000E0000000000000000000000000000000000010
:1000F0000000000000000000000000000000000000
:1001000000000000000000000000000000000000EF
:1001100000000000000000000000000000000000DF
:1001200000000000000000000000000000000000CF
:1001300000000000000000000000000000000000BF
:1001400000000000000000000000000000000000AF
:10015000000000000000000000000000000000009F
:10016000000000000000000000000000000000008F
:10017000000000000000000000000000000000007F
:10018000000000000000000000000000000000006F
:10019000000000000000000000000000000000005F
:1001A000000000000000000000000000000000004F
:1001B000000000000000000000000000000000003F
:1001C000000000000000000000000000000000002F
:1001D000000000000000000000000000000000001F
:1001E000000000000000000000000000000000000F
:1001F00000000000000000000000000000000000FF
:1002000001010101010101010101010101010101DE
:1002100001010101010101010101010101010101CE
:1002200001010101010101010101010101010101BE
:1002300001010101000101010101010101010101AF
:1002400001010101010101010001000101010101A0
:10025000010101010101010101010101010101008F
:10026000010101010101010101010001010101017F
:100270000101000101010101010001010001010072
:10028000010101010101010101010001010101015F
:100290000101010001010101000100010001010053
:1002A000010101010101010101010001010101013F
:1002B0000101010001010001010101000101010032
:1002C000010101010101010101010101010101001F
:1002D000010101010101010101010101010101010E
:1002E000000000000000000000000000000000000E
:1002F00000000000000000000000000000000000FE
:1003000001010101010101010101010101010101DD
:1003100001010101010101010101010101010101CD
:1003200001010101010101010100000101010101BF
:1003300001010001010001010100010100010100B2
:10034000010101010101010101000001010101019F
:100350000101010001000101000100010001010093
:10036000010101010101010101000001010101017F
:100370000101010001000001010101000101010072
:10038000010101010101010101010001010101005F
:100390000101000101000101010001010001010151
:1003A000010101010101010101010001010101003F
:1003B0000101010001000101000100010001010132
:1003C000010101010101010101010001010101001F
:1003D0000101010001000001010101000101010111
:1003E000000000000000000000000000000000000D
:1003F00000000000000000000000000000000000FD
:1004000001010101010101010101010101010101DC
:1004100001010101010101010101010101010101CC
:1004200001010001000101000101010101010101BF
:1004300000010101010101010100010101010101AE
:10044000010101000001010101010101010101019E
:10045000010100010101010101010101010101018D
:10046000010101010001010101010101010101017D
:10047000010100010101010100010101010101016E
:10048000010101010001000101010101010101015E
:10049000010100010101010101010101010101014D
:1004A000000000000000000000000000000000004C
:1004B000000000000000000000000000000000003C
:1004C000000000000000000000000000000000002C
:1004D000000000000000000000000000000000001C
:1004E000000000000000000000000000000000000C
:1004F00000000000000000000000000000000000FC
:1005000001010101010101010101010101010101DB
:1005100001010101010101010101010101010101CB
:1005200001010001000101000101010100010101BF
:1005300001010101010101010100010101010101AC
:10054000010101000001010101010101010101019D
:10055000010101010101000101010101010101018C
:10056000010101010001010101010101010101017C
:10057000010101010101000100010101010101016D
:10058000010101010001000101010101010101015D
:10059000010101010101000101010101010101014C
:1005A000000000000000000000000000000000004B
:1005B000000000000000000000000000000000003B
:1005C000000000000000000000000000000000002B
:1005D000000000000000000000000000000000001B
:1005E000000000000000000000000000000000000B
:1005F00000000000000000000000000000000000FB
:1006000001010101010101010101010101010101DA
:1006100001010101010101010101010101010101CA
:1006200000010001000101000101010101010101BE
:1006300001010101010101010100010101010101AB
:10064000010101000001010101010101010101019C
:10065000010101010101010101010001010101018B
:10066000010101010001010101010101010101017B
:10067000010101010101010100010001010101016C
:10068000010101010001000101010101010101015C
:10069000010101010101010101010001010101014B
:1006A000000000000000000000000000000000004A
:1006B000000000000000000000000000000000003A
:1006C000000000000000000000000000000000002A
:1006D000000000000000000000000000000000001A
:1006E000000000000000000000000000000000000A
:1006F00000000000000000000000000000000000FA
:1007000001010101010101010101010101010101D9
:1007100001010101010101010101010101010101C9
:1007200001010101010101010101010101010101B9
:1007300001010101010101010100010101000101AB
:100740000101010101010101010101010101010199
:10075000010101010101010001000101010101018B
:100760000101010101010101010101010101010179
:10077000010101000101010101000100010101016C
:100780000000000000000000000000000000000069
:100790000000000000000000000000000000000059
:1007A0000000000000000000000000000000000049
:1007B0000000000000000000000000000000000039
:1007C0000000000000000000000000000000000029
:1007D0000000000000000000000000000000000019
:1007E0000000000000000000000000000000000009
:1007F00000000000000000000000000000000000F9
:1008000000000100010101000000000000000000E4
:1008100000000000000000000000000000000000D8
:1008200000000000000000000000000000000000C8
:1008300000000000000000000000000000000000B8
:1008400000000000000000000101010101010101A0
:100850000101010101010101010101010101010188
:100860000101010101010101010101010101010178
:100870000101010101010101010101010101010168
:100880000101010101010101010101010101010158
:02089000010164
:00000001FF
